:020000040800F2
:100000002007002029020008C9110008A9100008D3
:10001000711100081F0400084913000800000000C7
:10002000000000000000000000000000CD110008EA
:100030005D04000800000000CB110008CF1100088B
:10004000430200084302000843020008430200087C
:10005000430200084302000843020008430200086C
:10006000430200084302000843020008430200085C
:10007000430200084302000843020008430200084C
:10008000430200084302000843020008430200083C
:10009000430200084302000843020008430200082C
:1000A000430200084302000843020008430200081C
:1000B000430200084302000843020008430200080C
:1000C00043020008430200084302000843020008FC
:1000D00043020008430200084302000843020008EC
:1000E00043020008430200084302000843020008DC
:1000F00043020008430200084302000843020008CC
:1001000043020008430200084302000843020008BB
:1001100043020008430200084302000843020008AB
:10012000430200084302000843020008430200089B
:10013000430200084302000843020008430200088B
:10014000430200084302000843020008430200087B
:10015000430200084302000843020008430200086B
:10016000430200084302000843020008430200085B
:100170004302000843020008430200080000000098
:10018000430200084302000800F002F800F03CF8C7
:100190000AA090E8000C82448344AAF10107DA45E2
:1001A00001D100F031F8AFF2090EBAE80F0013F0F8
:1001B000010F18BFFB1A43F001031847F0110000AC
:1001C00010120000103A24BF78C878C1FAD852073C
:1001D00024BF30C830C144BF04680C6070470000C1
:1001E0000023002400250026103A28BF78C1FBD840
:1001F000520728BF30C148BF0B6070471FB501F0E0
:10020000C8F81FBD10B510BD00F0CFF81146FFF7BC
:10021000F5FF01F0AAF800F0EDF803B4FFF7F2FFE4
:1002200003BC00F0F5F80000094880470948004782
:10023000FEE7FEE7FEE7FEE7FEE7FEE7FEE7FEE796
:10024000FEE7FEE704480549054A064B70470000F3
:100250006912000889010008200100202007002001
:10026000200300202003002053EA020C00F06980E4
:100270002DE9F04B4FF00006002B1FBFB3FA83F5BA
:1002800003FA05F424FA05F65E4012BF1643B2FAEB
:1002900082F502FA05F4C5F120051EBF22FA05FC1D
:1002A00044EA0C04203556EA044C4FEA144418BFC3
:1002B000641C4FF000084FF00009904271EB030CF2
:1002C00039D3002919BFB1FA81F701FA07F6B0FA5C
:1002D00080F700FA07F6C7F120071EBF20FA07FCD7
:1002E00046EA0C062037B6FBF4FCA7EB0507103FE7
:1002F00007F01F0BCBF120060CFA0BFB2CFA06F6CD
:1003000044BFB3460026202FA4BF5E464FF0000B2B
:100310005BEA060C08BF4FF0010B19EB0B09ABFBB6
:10032000027C48EB0608C01B06FB02CC0BFB03CC8F
:1003300071EB0C01C1E70B46024641464846BDE859
:10034000F08B13B54FF000004FF00001AFF30080C9
:10035000BDE81C4070474FF0000200B513469446BC
:100360009646203922BFA0E80C50A0E80C50B1F10D
:100370002001BFF4F7AF090728BFA0E80C5048BF21
:100380000CC05DF804EB890028BF40F8042B08BFBF
:10039000704748BF20F8022B11F0804F18BF00F8BB
:1003A000012B7047704770477047754600F02CF876
:1003B000AE4605006946534620F00700854618B052
:1003C00020B5FFF73FFFBDE820404FF000064FF09B
:1003D00000074FF000084FF0000B21F00701AC467A
:1003E000ACE8C009ACE8C009ACE8C009ACE8C00999
:1003F0008D46704710B50446AFF300802046BDE837
:100400001040FFF70ABF000000487047C0000020FE
:1004100001491820ABBEFEE7260002007047FEE748
:1004200010B5044800F058F9BDE810400221014819
:1004300000F017B81000002000B587B006AB0090A0
:1004400000200492039002900A466946024800F098
:100450001AF807B000BD000010000020704772B607
:10046000FEE790F82020012A07D0022A05D0416A31
:1004700041F48021416201207047006842690A43CB
:10048000426100207047F0B590F820500468A468DD
:10049000012D05D0022D03D0416A41F4802157E09F
:1004A00014F0406F01D1E5004FD5C4F3016401257C
:1004B000A5401D608D684FF4C0739DB1CE68354373
:1004C0004E6845EAC605066803EB0417F5514FF47C
:1004D000C275076805EB04150E697E51097D012977
:1004E00005D009E00E88CD6845EA4655EBE701687E
:1004F0004E5946F480764E511179D579567941EAB4
:10050000056195792D0445EA062529434FF4C67601
:10051000056806EB0416A9511178D57841EA056102
:10052000957852782D0445EA022211434FF4C475A0
:10053000026805EB04155151006803EB04114258A1
:1005400042F0010242500020F0BD416A41F4001126
:1005500041620120F0BD70B5040003D094F8200082
:1005600010B104E0012070BD204600F081F8206841
:10057000016841F00101016000F0E4F9054605263B
:1005800004E000F0DFF9401B0A2811D82068406819
:10059000C007F6D02068016821F00201016000F078
:1005A000D1F905460BE000F0CDF9401B0A2806D929
:1005B000606A40F40030606284F82060D2E720680E
:1005C00040688007EFD4207E0128206801683DD074
:1005D00021F080010160607E01282068016838D028
:1005E00021F040010160A07E01282068016833D01D
:1005F00021F020010160E07E0128206801682ED0F2
:1006000041F010010160207F01282068016829D095
:1006100021F008010160607F01282068016824D072
:1006200021F004010160D4E902010843D4E9041275
:10063000114308436168491E08432168C8610020CE
:100640006062012084F82000002070BD41F080012C
:10065000C0E741F04001C5E741F02001CAE721F0C1
:100660001001CFE741F00801D4E741F00401D9E7D8
:1006700010B586B0044614216846FFF76CFE134996
:10068000206888421FD112480021026842F000729F
:100690000260006800F0007005900D481038026894
:1006A00042F0080202600068022200F00800059093
:1006B0000320CDE90210CDE900020920049069462B
:1006C000044800F047F806B010BD00000064004088
:1006D00040380240000C024070B5044690F82000FB
:1006E000012804D0606A40F40020606218E0022013
:1006F00084F820002068016821F00101016000F009
:1007000021F905460EE000BF00F01CF9401B0A2845
:1007100008D9606A40F400306062052084F8200047
:10072000012070BD20684068C007EDD1606270BDD7
:1007300070B5044600F006F90546601C02D0044876
:100740000078044400F0FEF8401BA042FAD370BDCC
:10075000000000202DE9F84FDFF8BCA100220125A0
:1007600003264FF00F090AF1040BAAF1040E00BF93
:100770000B6805FA02F42340A34270D10F7907F009
:100780000307012F01D0022F16D187684FEA4208D4
:1007900006FA08FC27EA0C07D1F80CC00CFA08FC92
:1007A0004CEA070CC0F808C04768A7430C79C4F3AB
:1007B000001494403C4344600C79E443A4070AD0FD
:1007C000C4684FEA420C06FA0CF7BC438F6807FA7C
:1007D0000CF72743C7600C7904F00304022C12D1F4
:1007E000D40800EB840CDCF820405707FF0E09FA10
:1007F00007F824EA0804D1F8108008FA07F848EA54
:100800000408CCF8208004684FEA420C06FA0CF782
:10081000BC430F7907F0030707FA0CF7274307607B
:100820004C6814F4403F70D03C4C276847F4804734
:100830002760246822F0030704F480440094384CB5
:1008400007EB040CDCF8084897074FEA177809FA19
:1008500008F7BC43334FB84202D1002724E054E0EC
:10086000314FB84201D101271EE0304FB84201D1CB
:10087000022719E02E4FB84201D1032714E02D4F73
:10088000B84201D104270FE02B4FB84201D1052710
:100890000AE02A4FB84201D1062705E0284FB842A6
:1008A00001D1072700E0082707FA08F72743CCF80B
:1008B0000878DAF800405746D1F804C09C435FEA54
:1008C000CC2C00D51C433C60DBF800405F46D1F8DF
:1008D00004C09C435FEA8C2C00D51C433C60DEF8CE
:1008E00000407746D1F804C09C435FEA8C3C00D5B9
:1008F0001C433C60084F083F3C68D1F804C09C434F
:100900005FEACC3C00D51C433C60521C102AFFF42B
:100910002FAFBDE8F88F0000083C0140443802408A
:100920000030014000000240000402400008024084
:10093000000C024000100240001402400018024067
:10094000001C024001488068704700000000002041
:1009500002488168027811448160704700000020DD
:100960000B4810B5016841F400710160016841F461
:1009700080610160016841F480710160032000F032
:1009800061F80F2000F006F800F024F8002010BDF8
:10099000003C024070B50D4D04464FF47A71287842
:1009A000B1FBF0F00A490968B1FBF0F000F0DEFAA3
:1009B00048B9102C07D200222146501E00F022F820
:1009C00000206C6070BD012070BD000000000020A0
:1009D0000C0000200A4808B5016841F4804101601C
:1009E000006800F4804000900548001F016841F055
:1009F00080510160006800F08050009008BD000048
:100A000044380240F0B40E4B1B680C46C3F302237B
:100A1000C3F10705042D00D90425191D072901D2AA
:100A2000002300E0DB1E012606FA05F1491E2140E5
:100A300099409E40761E16403143F0BC00F085BCC4
:100A40000CED00E0064900F0070208684FF6FF03CE
:100A5000184040EA0220034A104308607047000033
:100A60000CED00E00000FA052DE9F0470E46050008
:100A700065D0DFF81481D8F80000F7B200F0070065
:100A8000B04207D288F80070D8F8000000F00700E4
:100A9000B04254D128683D4C810712D5400703D598
:100AA000206840F4E05020602878000703D52068D3
:100AB00040F4604020602068A96820F0F0000843FE
:100AC00020602878C0072DD030496868083901288F
:100AD00012D0022813D0032811D0096889070029F1
:100AE0002DDA216821F0030101432160FFF72AFF7D
:100AF000814641F2883A0EE009688903EFE7096808
:100B00008901ECE7FFF71EFFA0EB0901514502D96F
:100B10000320BDE8F0872068696800F00C00B0EBA6
:100B2000810FEFD1D8F80010404601F00701B14223
:100B300007D90770006800F00700B04201D001201B
:100B4000E7E72878400705D52068E96820F4E050F9
:100B5000084320602878000706D52068296920F41A
:100B6000604040EAC100206000F018F82168084A9F
:100B7000C1F30311515CC84006490860064800688B
:100B8000FFF708FF0020C4E7003C0240083802409D
:100B90009C1300080C00002004000020154810B52C
:100BA000006810F00C02144813D01449042A0FD026
:100BB000082A0ED10F4C241F2268236802F03F023E
:100BC0005B0207D52068C0F38810A0FB010106E096
:100BD000084610BD2168C1F38811A1FB0001002364
:100BE000FFF742FB2168C1F30141491C4900B0FBFA
:100BF000F1F010BD083802400024F40040787D0177
:100C00002DE9F84F04006ED02078DFF84C93C00730
:100C1000A9F104054AD009F104000168C1F381017A
:100C2000012908D00068C0F3810002280AD1D9F850
:100C30000000400206D52868800337D56068002888
:100C4000E1D033E06068B0F5803F10D0B0F5A02F60
:100C5000286810D020F480302860286820F4802094
:100C600028606068A8B1FFF76DFE06460DE02868B1
:100C700040F48030F4E740F480202860F7E700BFBC
:100C8000FFF760FE801B642873D828688003F7D5BF
:100C90000CE0FFF757FE064605E000BFFFF752FEE7
:100CA000801B6428F0D828688003F7D42078DFF808
:100CB000AC8280074FF0000A3ED5A748001D0168AE
:100CC00011F00C0F08D00068C0F3810002280BD18E
:100CD000D9F80000400207D42868800716D5E068DC
:100CE000012800D112E033E1E068B8B10120C8F872
:100CF0000000FFF727FE064605E000BFFFF722FED3
:100D0000801B0228C0D828688007F7D52868216989
:100D100020F0F80040EAC10028600DE0C8F800A00B
:100D2000FFF710FE064604E0FFF70CFE801B0228CA
:100D30001FD828688007F7D42078000722D5864F6F
:100D400087486169703771B101210160FFF7FAFDD1
:100D5000064604E0FFF7F6FD801B022809D8386834
:100D60008007F7D50EE0C0F800A0FFF7EBFD0646C0
:100D700005E082E0FFF7E6FD801B02287DD8386899
:100D80008007F7D42078400768D5DFF8CCB100277A
:100D90000BF13C0BDBF80000C0000BD4DBF80010BB
:100DA00041F08051CBF80010DBF80000012700F083
:100DB000805000906B4E3068C00510D4306840F40D
:100DC00080703060FFF7BEFD009005E0FFF7BAFDD0
:100DD0000099401A022850D83068C005F6D55E4EFA
:100DE000A0686C3601280FD00528306810D020F09C
:100DF00001003060306820F004003060A068B8B1B5
:100E0000FFF7A0FD00900FE0306840F00100F4E72C
:100E100040F004003060F7E7FFF794FD0099411AB5
:100E200041F28830814266D830688007F4D50EE000
:100E3000FFF788FD009007E0FFF784FD0099411A55
:100E400041F28830814256D830688007F4D42FB1FF
:100E5000DBF8001021F08051CBF80010A069C8B376
:100E60003D49091D0968C1F3810102294AD00228C0
:100E7000504607D0C8F8600000E03CE0FFF762FD94
:100E800004463BE04746C8F86000FFF75BFD0646B6
:100E900005E000BFFFF756FD801B02282BD828680D
:100EA0008001F7D4D4E907010843A16A2E4A490812
:100EB00002EB0141626A41EA8211084394F82C1066
:100EC00040EA0161C9F8001001203866FFF73AFDD9
:100ED000044606E03EE000BFFFF734FD001B022899
:100EE00009D828688001F7D534E000BFFFF72AFD54
:100EF000001B022802D90320BDE8F88F2868800172
:100F0000F4D427E00128F7D0D9F80000E26900F412
:100F1000800191421CD1226A00F03F01914217D119
:100F200047F6C071626A0140B1EB821F10D1A26A1C
:100F30004FF0FF3300F4403103EB5202B1EB024FAC
:100F400006D194F82C1000F07060B0EB016F01D066
:100F50000120D1E70020CFE70438024000004742DB
:100F6000800E4742007000400000FFFF10B5401E99
:100F7000B0F1807F01D3012010BD4FF0E02460610B
:100F80000F21601700F0E1F90020A0610720206127
:100F9000002010BD70B590F83C20012A32D0012409
:100FA00080F83C40022280F83D2003685A689D6822
:100FB00022F070060A6832435A60134B02689A4264
:100FC00014D0B2F1804F11D0104B9A420ED0104B7A
:100FD0009A420BD00F4B9A4208D00F4B9A4205D041
:100FE0000E4B9A4202D00E4B9A4204D1496825F02A
:100FF00080031943916080F83D40002180F83C1047
:10100000084670BD022070BD000001400004004091
:1010100000080040000C0040000401400040014076
:101020000018004010B5040003D094F83D0010B142
:1010300007E0012010BD002084F83C00204600F0AD
:101040001FF8022084F83D00211D206800F014F9EB
:10105000012084F8460084F83E0084F83F0084F8BC
:10106000400084F8410084F8420084F8430084F88A
:10107000440084F8450084F83D00002010BD0000C5
:1010800008B500680649884208D10648016841F061
:1010900010010160006800F01000009008BD000021
:1010A0000010004040380240FEE700000F4810B535
:1010B0000D4901600321416000214FF4202281602D
:1010C000C0E903124FF480124261017641768176C5
:1010D000C17601774177FFF73EFA002803D0BDE8DB
:1010E0001040FFF7BCB910BD0064004010000020A4
:1010F0000D4808B5016841F001010160016801F087
:1011000001010091016841F008010160016801F0EE
:1011100008010091016841F080010160006800F061
:101120008000009008BD0000303802401CB500244B
:101130000E4800940C4901940160A721C0E90114F4
:1011400063218461C160FFF76DFF08B1FFF787F984
:101150000094694605480194FFF71CFF002801D060
:10116000FFF77DF91CBD0000001000403800002092
:10117000FEE7000010B540210448FFF7ECF80348F3
:101180009FED030A80ED020A10BD000080000020E0
:10119000000000001CB50B494FF47A7008228883C8
:1011A00003208DF80000E8208DF8010000208DF864
:1011B00002008DF80300019069469001FFF73CF9A9
:1011C0001CBD000080000020FEE770477047FFF75D
:1011D000BFBB000030B593B030216846FFF7BBF8C5
:1011E00014210CA8FFF7B7F81D480025016841F04D
:1011F00080510160006800F080501190194801682A
:1012000041F4804101600068022400F480401190A4
:101210000120039010200490009406940820CDE94A
:101220000750A820CDE9090404200B906846FFF779
:10123000E7FC08B172B6FEE70CA90F2081E8310087
:101240004FF4A0500F904FF48050109005210CA83F
:10125000FFF70AFC002801D072B6FEE713B030BDDC
:1012600040380240007000400248016841F47001BB
:101270000160704788ED00E0F0B50268274B284D0B
:10128000284E294F294C4FF0804C984209D0604598
:1012900007D0A84205D0B04203D0B84201D0A04246
:1012A00004D122F0700E4A6842EA0E0298421BD026
:1012B000604519D0A84217D0B04215D0B84213D01B
:1012C000A04211D01A4DA8420ED01A4DA8420BD000
:1012D000194DA84208D0194DA84205D0184DA84272
:1012E00002D0184DA84203D122F44075CA682A439F
:1012F0004D6922F080022A438D68C5620D688562BF
:10130000984201D0A04201D109690163016841F00E
:1013100004010160012141610260F0BD0000014053
:101320000004004000080040000C004000040140A0
:1013300000400140004401400048014000180040C6
:10134000001C004000200040FEE70907090E0028AD
:1013500004DB00F1E02080F80014704700F00F007B
:1013600000F1E02080F8141D7047FFF7F9FAFFF74D
:1013700031FFFFF7BDFEFFF799FEFFF7D7FEFFF73E
:101380004FF8FFF7F7FEFFF705FF0520FFF7D0F94D
:10139000F9E74FF04070E1EE100A704700000000DE
:1013A000000000000102030406070809CC1300082E
:1013B0000000002010000000C4010008DC13000839
:1013C0001000002010070000E001000801000000EC
:0C13D00010000000000000000024F400E9
:040000050800018965
:00000001FF
